:100000000C9438000C9453000C9453000C9453003F
:100010000C9453000C9453000C9453000C94530014
:100020000C9453000C9453000C9453000C94530004
:100030000C9453000C9453000C9453000C945300F4
:100040000C9453000C94C1020C9453000C94530074
:100050000C94980F0C9453000C9453000C94530080
:100060000C9453000C9453000C9453000C945300C4
:1000700011241FBECFEFD4E0DEBFCDBF13E0A0E060
:10008000B1E0E4E2F4E202C005900D92AC36B107B3
:10009000D9F714E0ACE6B3E001C01D92A935B10771
:1000A000E1F70C9472000C940000CF93DF93CDB76E
:1000B000DEB7E4E3F0E08FEF8083EAE3F0E08EE286
:1000C0008083ABE3B0E0EBE3F0E0808182608C936F
:1000D000ABE3B0E0EBE3F0E0808180628C93DF91F2
:1000E000CF910895CF93DF93CDB7DEB70E9455002F
:1000F0000E94B2020E94960E7894A5E3B0E0E5E378
:10010000F0E0808181608C930E9485020E94FD0254
:100110000E9447030E9491030E94DB030E94250472
:100120000E946F040E94B9040E9403050E944D05BD
:100130000E9497050E940C0700C080916E038130D9
:1001400031F410926E030E9478110E948711809101
:100150007B038130E1F4A5E3B0E0E5E3F0E08081EA
:1001600084608C930E94A20D0E942A100E94AC070A
:100170000E94C1080E94F5090E9458060E943D078E
:10018000A5E3B0E0E5E3F0E080818B7F8C93809184
:100190006C03813091F610926C030E94E105CDCF83
:1001A000CF93DF93CDB7DEB764E084E00E94ED002B
:1001B0006CE480E00E94ED0010926E0380916E036B
:1001C0008823E1F36AE08CE60E94ED0060E085E0C0
:1001D0000E94ED00DF91CF910895CF93DF93CDB7CB
:1001E000DEB724970FB6F894DEBF0FBECDBF8B836A
:1001F0006C83ABE3B0E0EBE3F0E080818D7F8C9328
:1002000087E08A8340C0ABE3B0E0EBE3F0E08081BD
:10021000877F8C9300000000000000008A81282F57
:10022000332727FD309581E090E0022E02C0880F31
:10023000991F0A94E2F7982F8B81892389838981FA
:10024000882341F0ABE3B0E0EBE3F0E08081846031
:100250008C9307C0ABE3B0E0EBE3F0E080818B7FF1
:100260008C930000000000000000ABE3B0E0EBE383
:10027000F0E0808188608C930000000000000000A6
:100280008A8181508A838A8188230CF0BCCF87E0E1
:100290008A8340C0ABE3B0E0EBE3F0E08081877F8E
:1002A0008C9300000000000000008A81282F332773
:1002B00027FD309581E090E0022E02C0880F991F43
:1002C0000A94E2F7982F8C81892389838981882376
:1002D00041F0ABE3B0E0EBE3F0E0808184608C932D
:1002E00007C0ABE3B0E0EBE3F0E080818B7F8C9361
:1002F0000000000000000000ABE3B0E0EBE3F0E042
:10030000808188608C9300000000000000008A81DA
:1003100081508A838A8188230CF0BCCFABE3B0E0A4
:10032000EBE3F0E08081877F8C93ABE3B0E0EBE31D
:10033000F0E080818B7F8C93ABE3B0E0EBE3F0E007
:10034000808182608C9324960FB6F894DEBF0FBE36
:10035000CDBFDF91CF910895CF93DF93CDB7DEB7B7
:1003600024970FB6F894DEBF0FBECDBF8C83ABE3EE
:10037000B0E0EBE3F0E080818D7F8C9387E08A83AF
:100380004CC0ABE3B0E0EBE3F0E08081877F8C937F
:10039000000000000000000000000000000000005D
:1003A0008A81282F332727FD309581E090E0022EA7
:1003B00002C0880F991F0A94E2F7982F8C81892335
:1003C0008B838B81181644F4ABE3B0E0EBE3F0E0F1
:1003D000808184608C9307C0ABE3B0E0EBE3F0E096
:1003E00080818B7F8C9300000000000000000000E3
:1003F000000000000000ABE3B0E0EBE3F0E0808140
:1004000088608C93000000000000000000000000E5
:10041000000000008A8181508A838A8188230CF041
:10042000B0CF1B82ABE3B0E0EBE3F0E08081877FED
:100430008C9300000000000000000000000000009D
:10044000000087E08A833DC0ABE3B0E0EBE3F0E07F
:10045000808188608C93E9E3F0E0808189838981E1
:10046000992780719070181619068CF48A81282FAC
:10047000332727FD309581E090E0022E02C0880FDF
:10048000991F0A94E2F7982F8B81892B8B830000A8
:100490000000000000000000000000000000ABE3CE
:1004A000B0E0EBE3F0E08081877F8C9300000000F8
:1004B0000000000000000000000000008A81815060
:1004C0008A838A8188230CF0BFCFABE3B0E0EBE3F3
:1004D000F0E08081877F8C93ABE3B0E0EBE3F0E06A
:1004E00080818B7F8C93ABE3B0E0EBE3F0E0808125
:1004F00082608C938B81992724960FB6F894DEBF87
:100500000FBECDBFDF91CF910895CF93DF93CDB7CD
:10051000DEB70E94D00010926C0380916C03882398
:10052000E1F30E941E060E94C70B10926C0380919B
:100530006C038823E1F310926C0380916C03882391
:10054000E1F310926C0364E084E00E94ED006CE43F
:1005500080E00E94ED000E94E1050E947706DF9195
:10056000CF910895CF93DF93CDB7DEB7E3E5F0E009
:1005700082E08083E9E5F0E082E08083DF91CF9143
:1005800008951F920F920FB60F9211248F93CF935D
:10059000DF93CDB7DEB7809170038F5F80937003D8
:1005A00080917003883409F581E080936F03109285
:1005B0007003809114048F5F80931404809114045D
:1005C000843629F41092140481E080936C038091A6
:1005D00013048F5F80931304809113048A3029F4ED
:1005E0001092130481E080936E03DF91CF918F917D
:1005F0000F900FBE0F901F901895CF93DF93CDB73C
:10060000DEB762E480E00E94ED0010926C038091FE
:100610006C038823E1F310926C036AE989E00E947D
:10062000ED0010926E0380916E038823E1F3109227
:100630006E031092150416C080911504682F8AE08D
:100640000E94ED00809115049927FC01E95CFE4FA2
:100650008081682F8BE00E94ED00809115048F5FF0
:100660008093150480911504863330F360EA88E0A6
:100670000E94ED0010926E0380916E038823E1F3D7
:100680006CE480E00E94ED00DF91CF910895CF935C
:10069000DF93CDB7DEB762E480E00E94ED001092F8
:1006A0006C0380916C038823E1F310926C036BE977
:1006B00089E00E94ED0010926E0380916E03882302
:1006C000E1F310926E031092150416C08091150488
:1006D000682F8AE00E94ED00809115049927FC01A3
:1006E000E159FE4F8081682F8BE00E94ED008091E0
:1006F00015048F5F8093150480911504863330F3C1
:1007000060EA88E00E94ED0010926E0380916E0313
:100710008823E1F36CE480E00E94ED00DF91CF914B
:100720000895CF93DF93CDB7DEB762E480E00E94F7
:10073000ED0010926C0380916C038823E1F310921A
:100740006C036CE989E00E94ED0010926E038091C9
:100750006E038823E1F310926E031092150416C005
:1007600080911504682F8AE00E94ED0080911504A5
:100770009927FC01E955FE4F8081682F8BE00E948C
:10078000ED00809115048F5F80931504809115040E
:10079000863330F360EA88E00E94ED0010926E0329
:1007A00080916E038823E1F36CE480E00E94ED0009
:1007B000DF91CF910895CF93DF93CDB7DEB762E499
:1007C00080E00E94ED0010926C0380916C038823FE
:1007D000E1F310926C036DE989E00E94ED00109244
:1007E0006E0380916E038823E1F310926E031092E2
:1007F000150416C080911504682F8AE00E94ED0050
:10080000809115049927FC01E152FE4F8081682FE9
:100810008BE00E94ED00809115048F5F809315049A
:1008200080911504863330F360EA88E00E94ED0081
:1008300010926E0380916E038823E1F36CE480E0F4
:100840000E94ED00DF91CF910895CF93DF93CDB754
:10085000DEB762E480E00E94ED0010926C038091AC
:100860006C038823E1F310926C036EE989E00E9427
:10087000ED0010926E0380916E038823E1F31092D5
:100880006E031092150416C080911504682F8AE03B
:100890000E94ED00809115049927FC01E95EFD4F4F
:1008A0008081682F8BE00E94ED00809115048F5F9E
:1008B0008093150480911504863330F360EA88E054
:1008C0000E94ED0010926E0380916E038823E1F385
:1008D0006CE480E00E94ED00DF91CF910895CF930A
:1008E000DF93CDB7DEB762E480E00E94ED001092A6
:1008F0006C0380916C038823E1F310926C036FE921
:1009000089E00E94ED0010926E0380916E038823AF
:10091000E1F310926E031092150416C08091150435
:10092000682F8AE00E94ED00809115049927FC0150
:10093000E15BFD4F8081682F8BE00E94ED0080918C
:1009400015048F5F8093150480911504863330F36E
:1009500060EA88E00E94ED0010926E0380916E03C1
:100960008823E1F36CE480E00E94ED00DF91CF91F9
:100970000895CF93DF93CDB7DEB762E480E00E94A5
:10098000ED0010926C0380916C038823E1F31092C8
:100990006C0360EA89E00E94ED0010926E03809182
:1009A0006E038823E1F310926E031092150416C0B3
:1009B00080911504682F8AE00E94ED008091150453
:1009C0009927FC01E957FD4F8081682F8BE00E9439
:1009D000ED00809115048F5F8093150480911504BC
:1009E000863330F360EA88E00E94ED0010926E03D7
:1009F00080916E038823E1F36CE480E00E94ED00B7
:100A0000DF91CF910895CF93DF93CDB7DEB762E446
:100A100080E00E94ED0010926C0380916C038823AB
:100A2000E1F310926C0361EA89E00E94ED001092FC
:100A30006E0380916E038823E1F310926E0310928F
:100A4000150416C080911504682F8AE00E94ED00FD
:100A5000809115049927FC01E154FD4F8081682F96
:100A60008BE00E94ED00809115048F5F8093150448
:100A700080911504863330F360EA88E00E94ED002F
:100A800010926E0380916E038823E1F36CE480E0A2
:100A90000E94ED00DF91CF910895CF93DF93CDB702
:100AA000DEB762E480E00E94ED0010926C0380915A
:100AB0006C038823E1F310926C0362EA89E00E94E0
:100AC000ED0010926E0380916E038823E1F3109283
:100AD0006E031092150416C080911504682F8AE0E9
:100AE0000E94ED00809115049927FC01E950FD4F0B
:100AF0008081682F8BE00E94ED00809115048F5F4C
:100B00008093150480911504863330F360EA88E001
:100B10000E94ED0010926E0380916E038823E1F332
:100B20006CE480E00E94ED00DF91CF910895CF93B7
:100B3000DF93CDB7DEB762E480E00E94ED00109253
:100B40006C0380916C038823E1F310926C0363EAD9
:100B500089E00E94ED0010926E0380916E0388235D
:100B6000E1F310926E031092150416C080911504E3
:100B7000682F8AE00E94ED00809115049927FC01FE
:100B8000E15DFC4F8081682F8BE00E94ED00809139
:100B900015048F5F8093150480911504863330F31C
:100BA00060EA88E00E94ED0010926E0380916E036F
:100BB0008823E1F36CE480E00E94ED00DF91CF91A7
:100BC0000895CF93DF93CDB7DEB789ED80931504F9
:100BD00013C060E085E00E94ED0080911504682F4D
:100BE00086E00E94ED0064E587E00E94ED008091C0
:100BF00015048F5F80931504809115048C3D48F394
:100C000085EE8093150413C060E085E00E94ED003E
:100C100080911504682F86E00E94ED0064E587E06E
:100C20000E94ED00809115048F5F809315048091E0
:100C30001504883E48F3DF91CF910895CF93DF9359
:100C4000CDB7DEB764970FB6F894DEBF0FBECDBF49
:100C50008DE589838EE58A838FE58B8389E48C8398
:100C60008BE58D838DE18E838CE58F83188680E202
:100C7000898789E28A8786E38B8781E48C878AE08B
:100C80008D8781E48E8781E08F8786E2888B20E1E3
:100C9000CE010196AC0162E087E00E94A206649654
:100CA0000FB6F894DEBF0FBECDBFDF91CF91089590
:100CB000CF93DF93CDB7DEB760E085E00E94ED0013
:100CC0006FEC86E00E94ED006CE887E00E94ED008A
:100CD00061E085E00E94ED006BE086E00E94ED009F
:100CE0006DE887E00E94ED00DF91CF910895CF93EA
:100CF000DF93CDB7DEB760E085E00E94ED0060E2F3
:100D000086E00E94ED0060E887E00E94ED0060E070
:100D100085E00E94ED006EE386E00E94ED0064E84D
:100D200087E00E94ED0060E085E00E94ED006CE548
:100D300086E00E94ED0068E887E00E94ED00DF9108
:100D4000CF910895CF93DF93CDB7DEB72D970FB630
:100D5000F894DEBF0FBECDBF89876A875C874B875B
:100D60002D878A85282F33278EE190E0A901489F9F
:100D70009001499F300D589F300D11248985992786
:100D8000820F931F98878F838D85282F33278F811C
:100D90009885820F931F9E838D83109215048F81F7
:100DA00098859C838B8328C08B818A838B819C81CF
:100DB000892F99278983698185E00E94ED006A81E6
:100DC00086E00E94ED0040911504842F99279C0134
:100DD0008B859C85F901E80FF91F8081982F842F5E
:100DE0008F5F80931504692F87E00E94ED008B814F
:100DF0009C8101969C838B832B813C818D819E817C
:100E00002817390788F22D960FB6F894DEBF0FBE6B
:100E1000CDBFDF91CF910895CF93DF93CDB7DEB7EC
:100E200081E091E029E0AC016EE083E00E94A2063F
:100E3000DF91CF910895CF93DF93CDB7DEB722979F
:100E40000FB6F894DEBF0FBECDBF8A838A81882398
:100E500021F48A818652898303C08A8180538983E1
:100E60008981992787FD909522960FB6F894DEBF69
:100E70000FBECDBFDF91CF9108950F931F93CF93F6
:100E8000DF93CDB7DEB72D970FB6F894DEBF0FBE58
:100E9000CDBF80912204909123042EE130E0B9016E
:100EA0000E94EB11CB019B838A83CE0104962A8199
:100EB0003B814AE050E0BC01C9010E94BA11CE0159
:100EC0000496DC01FD0101900020E9F73197CF0184
:100ED0008A1B9B0B8983109215041CC080911504FA
:100EE000082F112780911504282F3327CE0104964F
:100EF000FC01E20FF31F80810E941B07282FCE0107
:100F00000996FC01E00FF11F2083809115048F5F8B
:100F10008093150480911504282F33278981992700
:100F200087FD909528173907CCF2298199818BE0AC
:100F3000382F391BCE010996AC016EE0832F0E9439
:100F4000A2062D960FB6F894DEBF0FBECDBFDF917F
:100F5000CF911F910F910895CF93DF93CDB7DEB757
:100F600029970FB6F894DEBF0FBECDBF80912A043B
:100F700090912B048E5590409C838B838B819C8118
:100F800023E030E0B9010E94EB11CB019A83898301
:100F900089819A818A30910524F089E090E09A83D2
:100FA000898389819A81992314F41A821982209164
:100FB00074033091750389819A818217930709F42C
:100FC000D7C089819A81823091052CF460E184E058
:100FD0000E94ED0004C060E084E00E94ED00898181
:100FE0009A81909375038093740380E88D8384E8DD
:100FF0008E8388E88F8389819A81998788878885FD
:1010000099858430910509F45FC08885998585307C
:101010009105DCF4888599858130910509F43FC0FC
:1010200088859985823091052CF48885998500976B
:1010300079F173C08885998582309105B9F18885E9
:10104000998583309105C9F168C088859985873075
:10105000910509F44EC088859985883091055CF426
:101060008885998585309105B1F188859985863087
:101070009105C1F152C0888599858830910509F4A0
:101080003FC0888599858930910509F440C045C0E5
:1010900080E88D8384E88E8388E88F833EC081E872
:1010A0008D8384E88E8388E88F8337C082E88D83C0
:1010B00084E88E8388E88F8330C083E88D8384E85A
:1010C0008E8388E88F8329C083E88D8385E88E83AB
:1010D00088E88F8322C083E88D8386E88E8388E842
:1010E0008F831BC083E88D8387E88E8388E88F8396
:1010F00014C083E88D8387E88E8389E88F830DC0D1
:1011000083E88D8387E88E838AE88F8306C083E82F
:101110008D8387E88E838BE88F8360E085E00E9473
:10112000ED0060E286E00E94ED008D81682F87E08F
:101130000E94ED0060E085E00E94ED006EE386E035
:101140000E94ED008E81682F87E00E94ED0060E034
:1011500085E00E94ED006CE586E00E94ED008F8145
:10116000682F87E00E94ED0060E084E00E94ED00BF
:1011700029960FB6F894DEBF0FBECDBFDF91CF9199
:101180000895CF93DF93CDB7DEB726970FB6F894C7
:10119000DEBF0FBECDBF80911A0490911B0426E1E3
:1011A00030E0B9010E94EB11CB0106969E838D833E
:1011B0008D819E8199230CF446C08D819E812AE009
:1011C00030E0B9010E94EB11CB018A838D819E81B1
:1011D0002AE030E0B9010E94EB118983898186956C
:1011E0008C5F89838A81282F332786E890E0821BD1
:1011F000930B9C838B8320910D0130910E018B8189
:101200009C818217930761F080910D0190910E01EE
:101210000E947A098B819C8169810E94B4090AC06D
:10122000909179038981981729F08B819C8169813C
:101230000E94B4098981809379038B819C8190936A
:101240000E0180930D018D819E8199230CF049C080
:101250008D819E81909581959F4F9E838D838D81F9
:101260009E812AE030E0B9010E94EB11CB018A8314
:101270008D819E812AE030E0B9010E94EB118983C3
:101280008981869589838A8199278A579F4F9C8374
:101290008B8320910D0130910E018B819C818217EF
:1012A000930761F080910D0190910E010E947A09DF
:1012B0008B819C8169810E94B4090AC09091790355
:1012C0008981981729F08B819C8169810E94B409DA
:1012D0008981809379038B819C8190930E01809307
:1012E0000D0126960FB6F894DEBF0FBECDBFDF917D
:1012F000CF910895CF93DF93CDB7DEB726970FB682
:10130000F894DEBF0FBECDBF9E838D831C821B82EF
:101310001DC08D818A838D819E81892F9927898324
:10132000698185E00E94ED006A8186E00E94ED00FF
:1013300060E087E00E94ED008D819E814E969E8345
:101340008D838B819C8101969C838B838B819C8177
:1013500088309105F0F226960FB6F894DEBF0FBEE6
:10136000CDBFDF91CF910895CF93DF93CDB7DEB797
:1013700027970FB6F894DEBF0FBECDBF9E838D8337
:101380006F831C821B8223C08D818A838D819E8105
:10139000892F99278983698185E00E94ED006A8100
:1013A00086E00E94ED008F819927FC01E35DFE4FEE
:1013B0008081682F87E00E94ED008D819E814E968E
:1013C0009E838D838B819C8101969C838B838B81F3
:1013D0009C8188309105C0F227960FB6F894DEBF45
:1013E0000FBECDBFDF91CF910895CF93DF93CDB7DF
:1013F000DEB726970FB6F894DEBF0FBECDBF809143
:1014000018049091190426E130E0B9010E94EB1113
:10141000CB019E838D838D819E8199230CF452C0D4
:101420008D819E812AE030E0B9010E94EB11CB0151
:101430008A838D819E812AE030E0B9010E94EB1100
:1014400089838981869589838A81282F332787E03C
:1014500090E0AC01421B530B9A018EE190E0AC018D
:10146000249FC001259F900D349F900D11240A9652
:101470009C838B8320910B0130910C018B819C818B
:101480008217930761F080910B0190910C010E94EB
:10149000C50A8B819C8169810E94280B0AC09091AA
:1014A00078038981981729F08B819C8169810E943A
:1014B000280B8981809378038B819C8190930C0108
:1014C00080930B018D819E8199230CF055C08D81F5
:1014D0009E81909581959F4F9E838D838D819E8166
:1014E0002AE030E0B9010E94EB11CB018A838D81A3
:1014F0009E812AE030E0B9010E94EB118983898145
:1015000086958C5F89838A81282F33278EE190E02E
:10151000AC01249FC001259F900D349F900D112494
:1015200086509F4F9C838B8320910B0130910C013F
:101530008B819C818217930761F080910B019091C0
:101540000C010E94C50A8B819C8169810E94280B35
:101550000AC0909178038981981729F08B819C812A
:1015600069810E94280B8981809378038B819C81FB
:1015700090930C0180930B0126960FB6F894DEBF72
:101580000FBECDBFDF91CF910895CF93DF93CDB73D
:10159000DEB726970FB6F894DEBF0FBECDBF9E8391
:1015A0008D838D819E819C838B8318C08B818A83E0
:1015B0008B819C81892F99278983698185E00E948D
:1015C000ED006A8186E00E94ED0060E087E00E9405
:1015D000ED008B819C8101969C838B838D819E8104
:1015E0009C01275F3F4F8B819C8182179307F0F20C
:1015F00080917803282F3327C901880F991F820F04
:10160000931FFC01EF5EFE4F80818823C1F08D8126
:101610009E8182969C838B838B818A838B819C8124
:10162000892F99278983698185E00E94ED006A816D
:1016300086E00E94ED0060E087E00E94ED002696C3
:101640000FB6F894DEBF0FBECDBFDF91CF910895E6
:10165000CF93DF93CDB7DEB727970FB6F894DEBFF1
:101660000FBECDBF9E838D836F838D819E819C83B2
:101670008B8324C08B8189838B819C81892F9927BF
:101680008A836A8185E00E94ED00698186E00E947C
:10169000ED008F81282F3327C901880F991F820FF2
:1016A000931FFC01E15FFE4F8081682F87E00E945D
:1016B000ED008B819C8101969C838B838D819E8123
:1016C0009C01275F3F4F8B819C818217930790F28B
:1016D0008D819E8104969C838B838B8189838B81F2
:1016E0009C81892F99278A836A8185E00E94ED0079
:1016F000698186E00E94ED008F81282F3327C90180
:10170000880F991F820F931FFC01E05FFE4F8081BD
:10171000682F87E00E94ED008F81282F3327C901B1
:10172000880F991F820F931FFC01EF5EFE4F80818F
:10173000882321F18D819E8182969C838B838B816E
:1017400089838B819C81892F99278A836A8185E08F
:101750000E94ED00698186E00E94ED008F81282FB4
:101760003327C901880F991F820F931FFC01EF5E79
:10177000FE4F8081682F87E00E94ED0027960FB60C
:10178000F894DEBF0FBECDBFDF91CF910895CF9308
:10179000DF93CDB7DEB760E085E00E94ED0063E83F
:1017A00086E00E94ED0060E987E00E94ED0060E0C5
:1017B00085E00E94ED0064E886E00E94ED0061E9AA
:1017C00087E00E94ED0060E085E00E94ED0065E8A2
:1017D00086E00E94ED0062E987E00E94ED0060E093
:1017E00085E00E94ED0066E886E00E94ED0063E976
:1017F00087E00E94ED0060E085E00E94ED0067E870
:1018000086E00E94ED0064E987E00E94ED0060E060
:1018100085E00E94ED0068E886E00E94ED0065E941
:1018200087E00E94ED0060E085E00E94ED0069E83D
:1018300086E00E94ED0066E987E00E94ED0060E02E
:1018400085E00E94ED006AE886E00E94ED0067E90D
:1018500087E00E94ED0060E085E00E94ED0061EA13
:1018600086E00E94ED0068E987E00E94ED0060E0FC
:1018700085E00E94ED0062EA86E00E94ED0069E9E1
:1018800087E00E94ED0060E085E00E94ED0063EAE1
:1018900086E00E94ED006AE987E00E94ED0060E0CA
:1018A00085E00E94ED0064EA86E00E94ED006BE9AD
:1018B00087E00E94ED0060E085E00E94ED0065EAAF
:1018C00086E00E94ED006CE987E00E94ED0060E098
:1018D00085E00E94ED0066EA86E00E94ED006DE979
:1018E00087E00E94ED0060E085E00E94ED0067EA7D
:1018F00086E00E94ED006EE987E00E94ED0060E066
:1019000085E00E94ED0068EA86E00E94ED006FE944
:1019100087E00E94ED0060E085E00E94ED006FEB43
:1019200086E00E94ED0060EA87E00E94ED0060E042
:1019300085E00E94ED0060EC86E00E94ED0061EA27
:1019400087E00E94ED0060E085E00E94ED0061EC20
:1019500086E00E94ED0062EA87E00E94ED0060E010
:1019600085E00E94ED0062EC86E00E94ED0063EAF3
:1019700087E00E94ED0060E085E00E94ED0063ECEE
:1019800086E00E94ED0064EA87E00E94ED0060E0DE
:1019900085E00E94ED0064EC86E00E94ED0065EABF
:1019A00087E00E94ED0060E085E00E94ED0065ECBC
:1019B00086E00E94ED0066EA87E00E94ED0060E0AC
:1019C00085E00E94ED0066EC86E00E94ED0067EA8B
:1019D00087E00E94ED0060E085E00E94ED006DED83
:1019E00086E00E94ED0068EA87E00E94ED0060E07A
:1019F00085E00E94ED006EED86E00E94ED0069EA50
:101A000087E00E94ED0060E085E00E94ED006FED50
:101A100086E00E94ED006AEA87E00E94ED0060E047
:101A200085E00E94ED0060EE86E00E94ED006BEA2A
:101A300087E00E94ED0060E085E00E94ED0061EE2D
:101A400086E00E94ED006CEA87E00E94ED0060E015
:101A500085E00E94ED0062EE86E00E94ED006DEAF6
:101A600087E00E94ED0060E085E00E94ED0063EEFB
:101A700086E00E94ED006EEA87E00E94ED0060E0E3
:101A800085E00E94ED0064EE86E00E94ED006FEAC2
:101A900087E00E94ED0060E085E00E94ED006BEFC2
:101AA00086E00E94ED0060EB87E00E94ED0060E0C0
:101AB00085E00E94ED006CEF86E00E94ED0061EB96
:101AC00087E00E94ED0060E085E00E94ED006DEF90
:101AD00086E00E94ED0062EB87E00E94ED0060E08E
:101AE00085E00E94ED006EEF86E00E94ED0063EB62
:101AF00087E00E94ED0060E085E00E94ED006FEF5E
:101B000086E00E94ED0064EB87E00E94ED0061E05A
:101B100085E00E94ED0060E086E00E94ED0065EB4C
:101B200087E00E94ED0061E085E00E94ED0061E049
:101B300086E00E94ED0066EB87E00E94ED00DF91F9
:101B4000CF910895CF93DF93CDB7DEB764970FB6EB
:101B5000F894DEBF0FBECDBF83E090E09C8B8B8BF3
:101B60001A82198283E990E09C838B8310927B0315
:101B7000CFC08B899C89FC01E458FC4F8081992758
:101B8000CD979A8B898B8B899C8901969C8B8B8BAB
:101B90008B899C89FC01E458FC4F80819927CD9763
:101BA000988B8F878B899C8901969C8B8B8B8B89DB
:101BB0009C89FC01E458FC4F80819927CD979E8732
:101BC0008D878B899C8901969C8B8B8B8B899C89BB
:101BD000FC01E458FC4F80819927CD979C878B8727
:101BE0008B899C8901969C8B8B8B89899A899C0116
:101BF000220F331F220F331F8F8598899595879564
:101C0000959587959595879595958795822B932B97
:101C10009A8789878F8598898F7090709C0122950B
:101C20003295307F3227207F32278D859E8595958E
:101C3000879595958795822B932B98878F838D8594
:101C40009E85837090709C0100243695279507949B
:101C5000369527950794322F202D8B859C85822BD6
:101C6000932B9E838D838B819C8101979C838B8397
:101C70008B819C812FEF8F3F920709F44EC08981A1
:101C80009A819C018091670390916803F901E80FA4
:101C9000F91F8985808389819A8101969A83898336
:101CA0008B819C8101979C838B838B819C812FEFFF
:101CB0008F3F920791F189819A819C0180916703FE
:101CC00090916803F901E80FF91F8F818083898162
:101CD0009A8101969A8389838B819C8101979C8349
:101CE0008B838B819C812FEF8F3F9207B1F089818D
:101CF0009A819C018091670390916803F901E80F34
:101D0000F91F8D81808389819A8101969A838983C5
:101D10008B819C81009709F02CCF64960FB6F894C4
:101D2000DEBF0FBECDBFDF91CF910895CF93DF937C
:101D3000CDB7DEB7E9E2F0E082E28083E0E4F0E0F4
:101D40001082E0E2F0E082E28083ECE5F0E01082D5
:101D5000A2E3B0E0E2E3F0E0808181608C93A8E34D
:101D6000B0E0E8E3F0E0808184608C93EAE2F0E0A8
:101D700088E98083E0E4F0E086E88083EBE2F0E04D
:101D800082EC8083E1E2F0E088E98083ECE5F0E03A
:101D900086E88083E2E2F0E082EC8083DF91CF91FD
:101DA0000895CF93DF93CDB7DEB721970FB6F894A0
:101DB000DEBF0FBECDBF8983EBE2F0E080819927C3
:101DC000807290700097C1F3ECE2F0E0898180832B
:101DD00021960FB6F894DEBF0FBECDBFDF91CF9135
:101DE0000895CF93DF93CDB7DEB726970FB6F8945B
:101DF000DEBF0FBECDBF9E838D838D819E81DC01B2
:101E0000FD0101900020E9F73197CF018A1B9B0B60
:101E10009C838B831A8219820FC029813A818D811C
:101E20009E81F901E80FF91F80810E94D10E8981FE
:101E30009A8101969A83898329813A818B819C8139
:101E40008217930750F7809169030E94D10E809109
:101E50006A030E94D10E26960FB6F894DEBF0FBE1D
:101E6000CDBFDF91CF910895CF93DF93CDB7DEB78C
:101E700066970FB6F894DEBF0FBECDBF9E8B8D8BDD
:101E80008D899E894AE050E09E012F5F3F4FB90146
:101E90000E94BA11CE0101960E94F10E66960FB60D
:101EA000F894DEBF0FBECDBFDF91CF910895CF93E1
:101EB000DF93CDB7DEB722970FB6F894DEBF0FBE23
:101EC000CDBF8A8387E089831FC08A81482F552729
:101ED0008981282F332727FD309581E090E0022E5D
:101EE00002C0880F991F0A94E2F7842395231816DD
:101EF000190624F481E30E94D10E03C080E30E94FE
:101F0000D10E89818150898389818823F4F680915B
:101F100069030E94D10E80916A030E94D10E22961D
:101F20000FB6F894DEBF0FBECDBFDF91CF910895FD
:101F30001F920F920FB60F9211242F933F938F93FE
:101F40009F93AF93BF93EF93FF93CF93DF93CDB75F
:101F5000DEB72297DEBFCDBFE3E2F0E08081809361
:101F60005804809158048D30D1F480917A038130E7
:101F7000B1F4A5E3B0E0E5E3F0E08081877F8C93E6
:101F800010927A0381E080937B0380911204992759
:101F900020915804FC01E458FC4F208348C08091F4
:101FA0007A03282F33273A83298389819A810097DE
:101FB00031F029813A812130310521F138C08091F9
:101FC0005804833271F480917B03882351F481E0BB
:101FD00080937A03A5E3B0E0E5E3F0E080818860D8
:101FE0008C931092120430911204832F9927209120
:101FF0005804FC01E458FC4F2083832F8F5F8093AB
:10200000120415C080911204992720915804FC01F4
:10201000E458FC4F208380911204863930F480917B
:1020200012048F5F8093120402C010927A032296EA
:10203000F894DEBFCDBFDF91CF91FF91EF91BF91BB
:10204000AF919F918F913F912F910F900FBE0F9065
:102050001F901895CF93DF93CDB7DEB76E970FB66D
:10206000F894DEBF0FBECDBF209118043091190443
:10207000CE010B964AE050E0BC01C9010E94BA11A2
:1020800080E4898384E48A8380E38B831C82CE018D
:102090000B96DC01FD0101900020E9F73197CF019B
:1020A0008A1B9B0B9E01255F3F4FAC01B901CE01FE
:1020B00001960E94AA11CE010196DC01FD0101905A
:1020C0000020E9F731979F012A1B3B0BCE010196B7
:1020D000820F931FFC0183E290E091838083CE0105
:1020E00001960E94F10E20911A0430911B04CE013A
:1020F0000B964AE050E0BC01C9010E94BA1180E48D
:10210000898384E48A8381E38B831C82CE010B96CE
:10211000DC01FD0101900020E9F73197CF018A1B16
:102120009B0B9E01255F3F4FAC01B901CE0101968B
:102130000E94AA11CE010196DC01FD010190002050
:10214000E9F731979F012A1B3B0BCE010196820FC5
:10215000931FFC0183E290E091838083CE0101967E
:102160000E94F10E2091220430912304CE010B969F
:102170004AE050E0BC01C9010E94BA1180E48983A1
:1021800088E68A838DE38B831C82CE010B96DC016B
:10219000FD0101900020E9F73197CF018A1B9B0BCD
:1021A0009E01255F3F4FAC01B901CE0101960E940F
:1021B000AA11CE010196DC01FD0101900020E9F792
:1021C00031979F012A1B3B0BCE010196820F931F73
:1021D000FC0183E290E091838083CE0101960E940E
:1021E000F10E20912A0430912B04CE010B964AE087
:1021F00050E0BC01C9010E94BA1180E4898386E5E0
:102200008A838CE68B831C82CE010B96DC01FD0158
:1022100001900020E9F73197CF018A1B9B0B9E01AB
:10222000255F3F4FAC01B901CE0101960E94AA1172
:10223000CE010196DC01FD0101900020E9F7319704
:102240009F012A1B3B0BCE010196820F931FFC01BD
:1022500083E290E091838083CE0101960E94F10E8B
:102260002091740330917503CE010B964AE050E043
:10227000BC01C9010E94BA1180E4898386E58A8382
:1022800081E48B831C82CE010B96DC01FD01019061
:102290000020E9F73197CF018A1B9B0B9E01255F38
:1022A0003F4FAC01B901CE0101960E94AA11CE01A7
:1022B0000196DC01FD0101900020E9F731979F01B3
:1022C0002A1B3B0BCE010196820F931FFC0183E278
:1022D00090E091838083CE0101960E94F10E6E966C
:1022E0000FB6F894DEBF0FBECDBFDF91CF9108953A
:1022F000CF93DF93CDB7DEB7A5E3B0E0E5E3F0E041
:10230000908182E089278C93DF91CF910895CF93BC
:10231000DF93CDB7DEB7809173038130C1F4809134
:102320007203813051F4A5E3B0E0E5E3F0E0808191
:102330008E7F8C93109272030AC0A5E3B0E0E5E3B0
:10234000F0E0808181608C9381E080937203DF9163
:10235000CF910895FB01DC010D900020E9F7119762
:102360004150504028F0019000200D92C9F7089587
:102370001C920895FB019F01E8944230C4F045325D
:10238000B4F44A3029F497FB1EF4909581959F4F41
:10239000642F77270E94FE11805D8A330CF0895DDF
:1023A0008193CB010097A1F716F45DE2519310825F
:1023B000C9010C94DB11DC01FC0101900020E9F75C
:1023C0003297AE17BF0730F47C91608170833197EC
:1023D0006D93F7CF089597FB092E07260AD077FD56
:1023E00004D00CD006D000201AF4709561957F4F70
:1023F0000895F6F7909581959F4F0895AA1BBB1BF2
:1024000051E107C0AA1FBB1FA617B70710F0A61BF4
:10241000B70B881F991F5A95A9F780959095BC0115
:04242000CD0108954D
:1024240001125A2C294400000A31002300230054CD
:1024340064665363655262005161005060005060ED
:1024440000516100526200536365546466676869B1
:102454006A6B6B6A6968671A440592820A91A0AA3A
:10246400A466AA691AAA196AAA02AAAA86AAAA6AC0
:10247400AAAA6AAAAAAAAAAAAAAAAAAAAAA8AAAAFA
:10248400A4AAAAA1AAAA91AAAA85AAAA4555556A44
:10249400A555AA9155AA4555AA1555A91555A8504B
:1024A40000A44000A1000090000080000050000043
:1024B4001000005000685000A85000A95400AA540D
:1024C40000AA5500AA5555555A91554AA5554AAAE8
:1024D400554AAA554AAA154AAA054AAA014AAA006F
:1024E4004AAA0046AA0011AA00151A0015410015AF
:1024F40054001555005555405555415554555546AC
:10250400826AAA0AAAAA1A41AA5609AAA914AAA9B5
:1025140068AAAA56AAAAA6AAAAA8AAAAA8AAAAAAB5
:10252400AAAAAAAAAAAA1AAAAA42AAAA546AAA55EA
:1025340006AA00006A5555A451A9A9146AAA452AF5
:102544002A854A2AA1466AA452A1A91441AA1404BC
:102554002A45292A856AAA91AAAAA1AAAAA4AAAA4A
:10256400A8AAAAA9AAAAA9AAAAAAAAAAAA5555150A
:102574005555155555855555915555A15555A45540
:1025840055A855556915552A15551A45554A855561
:102594004A955556915552A15551A55515A4551412
:1025A400A85554A85555555569155469515469523F
:1025B40054A85254A85654A85655A85655A856552A
:1025C400A85655A85655A85655A85654A85654A8C2
:1025D4005654A8525469525469515569155555AA0F
:1025E400AAAAAAAAAAAAAAAAAAAA90AAAA95AAAA76
:1025F40095AAAA95AAAA95AAAA95AAAA95AAAA95B5
:10260400AAAA95AAAA95AAAA95AAAA91AAAAA4AA84
:10261400AAA9AAAAAA5555AAAA15AAA955AAA45507
:10262400000155555000550000540000540000505E
:10263400000050000150001A50002A5000155000AC
:10264400005000005400000500009040005555550E
:1026540040AA5554AA55546A55546A15546A0554E7
:102664006A0141AA005AAA06AAAAAAAAAAAAAAAAB6
:10267400AAAAAA55556A00001A00554A00554601EF
:0C2684005556055552555516040D0A0018
:00000001FF
